:10000000C6EF03F000000000BBEF03F000000000AB
:0A0010000000000000000000F3D71C
:10001C00026A036A800E0318006E800E005C02E117
:10002C00080E025C11E28296800E0101D615016E5B
:10003C000150800A02E1828801D082988286D637EC
:0A004C00D691024A032AE6D71200FB
:1000560082928290D5C1D6F1DEDF070E0C6E7D0E40
:0E0066000D6E0D2EFED70C2EFCD782801200E0
:0E00740082828290D3C1D6F1CFDF828012004B
:10008200070E0101D415006E400E0010D56FE2DF9D
:100092007F0E0101D315006E800E0010D56FDADFDE
:0200A20012004A
:1000A400010E036E800E080A006E800E0318005CB9
:1000B40019E3819A800E0101CE15016E000ECEBFA8
:1000C400FF0E026E000E0216000E021802E1800EF0
:1000D400011802E1818001D08190CE37CE91818ACE
:0800E400032AE0D7818A120013
:0E00EC00ACB202D00000FCD7CEC1ADFF1200B6
:1000FA00056A066A076A086A0F0E046E800E0418FB
:10010A00006E800E000A005C24E3819A818A81A82D
:10011A001ED00404006E000E04BEFF0E016E000E17
:10012A00015A00C002F0010E006E000E016E02506C
:10013A0005E0003600900136FF0FFAD70050052679
:10014A0001500622000E01BEFF0E072208220406F5
:10015A00D5D705C000F006C001F007C002F008C0FC
:04016A0003F012008C
:10016E00CEC102F0CFC103F002C000F003C001F017
:10017E00024A032A00C0E9FF01C0EAFFEE5201E085
:10018E00F3D70101CE51025C006ECF510358016EC0
:0A019E00010E005E000E015A12006F
:1001A800086A096A100E0C6E0134083609360450C4
:1001B800085E0550D8A0053C095ED8B007D00450A9
:1001C80008260550D8B0053C0926D89000360136D7
:0601D8000C2EEAD7120014
:0A01DE00120E0D6E0D2EFED712005A
:1001E800200E0101CE5D04E3CE517F0801E301D06A
:1001F8001200050ECE03F3CF00F0F4CF01F0A00EED
:10020800005CCF6F000E0158D06F050ED16F000E45
:10021800D26F800E006E800ED219005C02E1D151BF
:10022800000818E24A0ECF25F66E0E0ED021F76EA2
:10023800000EF86E000ED0BFFF0EF8220900F5CFB1
:10024800D3F114DF0101CF4BD02B010ED15F000E8B
:0A025800D25BDFD7D36B0ADF120080
:100262000101D36BD46B0CDF0101CE6BCF6B800E1F
:10027200030A006E800ECF19005C02E1CE518008A5
:1002820010E3D36BF6DE040E0C6E3D0E0D6E0D2EDA
:10029200FED70C2EFCD7000000000101CE4BCF2B65
:0402A200E6D7120089
:1002A6008196210E0C6E760E0D6E0D2EFED70C2E3F
:1002B600FCD70000818A81868194040E0C6E3D0E67
:1002C6000D6E0D2EFED70C2EFCD70000000081808F
:1002D600040E0C6E3D0E0D6E0D2EFED70C2EFCD7A9
:1002E60000000000818A040E0C6E3D0E0D6E0D2E70
:1002F600FED70C2EFCD700000000010E0101C76FCF
:10030600000EC86F800E006E800EC819005C02E1F8
:10031600C751050809E3100ECE6FC1DEFF0ECE6F82
:10032600BEDEC74BC82BEED7100ECE6FB8DE040E5E
:100336000C6E3D0E0D6E0D2EFED70C2EFCD700005A
:100346000000CE6BACDE040E0C6E3D0E0D6E0D2E57
:10035600FED70C2EFCD700000000100ECE6F9FDEDD
:10036600040E0C6E3D0E0D6E0D2EFED70C2EFCD718
:1003760000000000540ECE6F92DE040E0C6E3D0E91
:100386000D6E0D2EFED70C2EFCD7000000001200BD
:10039600C26AC00EC212C18CC18EC7C100F000363F
:1003A600009000360090003600900050C212C280C5
:1003B60013DFC284C2A401D0FDD7C4CF01F0006A06
:0C03C600C3500012000E0112C290120081
:1003D2000101CB6B050ECB5D0AE2CB51C925E16E63
:1003E200000ECA21E26E200EE66ECB2BF3D7CB5164
:1003F200C925E16E000ECA21E26EE66ACB07CB5137
:10040200C925CC6F000ECA21CD6F0A0E046E000EF4
:10041200056EC7C100F0C8C101F0C5DE08C000F01A
:1004220009C001F0300E0026CCC1E1FFCDC1E2FFD0
:1004320000C0E6FF0A0E046E000E056EC7C100F092
:10044200C8C101F0B0DE00C0C7F101C0C8F1000EA2
:10045200011802E1000E001801E102D0CB07CFD74C
:02046200120086
:10046400A6A202D00000FCD7A69CC7C1A9FFC8C1A0
:10047400A8FFA69EA684F2CF00F0F29E550EA76EAA
:10048400AA0EA76EA68200BE02D0F29E01D0F28E02
:04049400A694120018
:100498003FC1CEF140C1CFF166DE00C0C8F1C76BE5
:1004A800C7513F25E96E000EC7BFFF0E4021EA6E17
:1004B800EECFC9F1BBA104D0C9C1CEF113DE03D080
:1004C800C9C1CEF18DDE0101C72B800EC719006EA0
:1004D800800EC819005CE4E319D029D028D02C0E6E
:1004E800CE6F00DE24D0090E0101CE6FFBDD1FD0D8
:1004F8000D0E0101CE6FF6DD0A0E0101CE6FF2DDA1
:1005080016D02A0E0101CE6FEDDD11D00101BB51CD
:10051800000AE3E0BB51010AE1E0BB51030ADFE056
:10052800BB51050AE0E0BB51070AE2E0EAD7120036
:100538000B6A0A6A096A00500402F4CF09F0F3CF83
:1005480008F001500502F4CF0BF0F3CF0AF0005089
:100558000502F3500926F4500A22E86A0B220150DA
:100568000402F3500926F4500A22E86A0B2208C054
:1005780000F009C001F00AC002F00BC003F012003D
:100588000A0E0101CE6FAEDD0D0E0101CE6FAADDA0
:0205980012004F
:10059A00C7C104F0C8C105F004C002F005C003F0E9
:1005AA00044A052AC9C100F0CAC101F00101C94BB8
:1005BA00CA2B00C0E9FF01C0EAFF02C0E1FF03C085
:1005CA00E2FFEECFE6FF02C0E9FF03C0EAFFEE5208
:0E05DA0001E0E2D7C7C100F0C8C101F0120075
:1005E800C7C104F0C8C105F004C0E9FF05C0EAFFAF
:1005F800EE5203E0044A052AF7D704C002F005C00A
:1006080003F0044A052AC9C100F0CAC101F001017A
:10061800C94BCA2B00C0E9FF01C0EAFF02C0E1FFD5
:1006280003C0E2FFEECFE6FF02C0E9FF03C0EAFF26
:10063800EE5201E0E2D7C7C100F0C8C101F01200D4
:0A064800000E9EBA010E006E1200B3
:10065200EC0E0101886F000E896FCE0E8A6F010EBB
:100662008B6FD20E846F060E856F000E866F000EA2
:10067200876F480E8C6F060E8D6F000E8E6F000E08
:100682008F6FFF0E936FFF0E946F000E956F000E2B
:10069200966FAC8A900EAB6E948E949C9EAA03D0F9
:0806A200AECF00F0FBD71200FF
:1006AA000900F5CFE6FF0006FBE10106F9E11200B9
:1006BA0081A201D0FDD781B201D0FDD7380E010148
:0806CA00CE6FEBDC15DD120020
:1006D200AECF92F1ABA202D0AB98AB8892C100F040
:0206E200120004
:1006E400A69CC7C1A9FFA69EA680A8CF00F01200B1
:1006F400828482808294030E0B6E8A0E0C6E550ED9
:100704000D6E0D2EFED70C2EFCD70B2EFAD7000043
:1007140000008284210E0101D56F9BDC900E010143
:10072400D56F97DC050E0101D56F93DC130E010123
:10073400D56F8FDC200E0101D56F8BDC210E0C6E82
:10074400760E0D6E0D2EFED70C2EFCD700000C0E6F
:100754000101D56F7EDC83DD410E0C6EEE0E0D6E55
:100764000D2EFED70C2EFCD70000D36BD46B87DC88
:02077400120071
:100776009EA008D00101904B912BFF0ECF6EFF0E6D
:06078600CE6E9E901100F2
:10078C00CDEC08F0816A120E936EF19EFF0E806E16
:10079C00010E926E010EC26E8E0EC16E946AD56AF7
:1007AC000A0EAF6EAC844FDF49DF0050010A03E143
:1007BC008ADF00C0BCF1070E0101BB6FDFDE3FC159
:1007CC00C7F140C1C8F1B10E0101C96F000ECA6F6B
:1007DC00DEDE00C03FF101C040F158DE3FC1C7F181
:1007EC0040C1C8F1A00E0101C96F000ECA6FCFDE67
:1007FC0000C03FF101C040F149DE9EC0CEF19FC068
:10080C00CFF1AFDC00C0C3F101C0C4F1C16BC26B4E
:10081C00C451C25D02E1C351C15D12E2C1C1C7F155
:10082C00C15100019E25E96E0101C25100019F21B9
:10083C00EA6EEECFC8F110DE0101C14BC22BE8D736
:10084C00C16BC26BC451C25D02E1C351C15D0EE20A
:10085C00C1C1C7F141DF00C0BFF1000EC06FBFC105
:10086C00CEF13EDC0101C14BC22BECD787DE3FC180
:10087C00C7F140C1C8F1C80E0101C96F000ECA6FA3
:10088C0086DE00C03FF101C040F100DE0101BB6B10
:10089C002BDF020E0B6E450E0C6EA90E0D6E0D2E7F
:1008AC00FED70C2EFCD70B2EFAD70000000001014E
:1008BC00D36BD46B41EC00F03FC1C7F140C1C8F120
:1008CC00F20E0101C96F000ECA6F61DE00C03FF16C
:1008DC0001C040F1DBDD819E0101D36BD46B41EC97
:1008EC0000F03FC1C7F140C1C8F1E10E0101C96F71
:1008FC00000ECA6F4CDE00C03FF101C040F1C6DDF6
:10090C000101D36B010ED46F41EC00F03FC1C7F174
:10091C0040C1C8F18D0E0101C96F000ECA6F37DEE0
:10092C0000C03FF101C040F1B1DD0101D36B020EFB
:10093C00D46F41EC00F03FC1C7F140C1C8F1370E94
:10094C000101C96F000ECA6F22DE00C03FF101C069
:10095C0040F19CDD0101D36B030ED46F41EC00F030
:10096C003FC1C7F140C1C8F1260E0101C96F000E8D
:10097C00CA6F0DDE00C03FF101C040F187DD0101FF
:10098C00D36B040ED46F41EC00F03FC1C7F140C1F2
:10099C00C8F1150E0101C96F000ECA6FF8DD00C059
:1009AC003FF101C040F172DD0101D36B050ED46F34
:1009BC0041EC00F03FC1C7F140C1C8F1480E010144
:1009CC00C96F000ECA6FE3DD00C03FF101C040F1FA
:1009DC005DDD0101D36B060ED46F41EC00F03FC11D
:1009EC00C7F140C1C8F17C0E0101C96F000ECA6F7E
:1009FC00CEDD00C03FF101C040F148DD0101D36BF9
:100A0C00070ED46F41EC00F03FC1C7F140C1C8F1F3
:100A1C006B0E0101C96F000ECA6FB9DD00C03FF14A
:100A2C0001C040F133DD010E0101BB6FA7DD35DCE8
:100A3C003FC1C7F140C1C8F1590EC96F000ECA6F52
:100A4C00A6DD00C03FF101C040F120DD97DD3FC1C4
:100A5C00C7F140C1C8F1060E0101C96F010ECA6F82
:100A6C0096DD00C03FF101C040F110DD87DD010EC5
:100A7C000101BB6FB96B800EB919006E800E100AA4
:100A8C00005C42E2B9C100F0000EB9BFFF0E016E6E
:100A9C00003600900136990E0024C56F010E01201E
:100AAC00C66FB9C100F0000EB9BFFF0E016ED60EB5
:100ABC00046E060E056E3ADD0D0E0026020E0122A6
:100ACC00C5C1E1FFC6C1E2FF00C0E6FF01C0E6FF01
:100ADC00B9C100F0000EB9BFFF0E016E00360090D8
:100AEC000136990E0024E96E010E0120EA6EEECF5C
:100AFC00C7F1EECFC8F13FC1C9F140C1CAF163DC07
:100B0C00C5DC0101B92BB7D739DD0D0E0B6EAF0E5D
:100B1C000C6EB60E0D6E0D2EFED70C2EFCD70B2EBA
:100B2C00FAD700000101B96BBC6BBD6BBE6B31EC2D
:100B3C0001F0010EBA6F82DD0050010A1DE1C3DD28
:100B4C0000C0BCF10AD00101BA7715D0BA7113D02C
:100B5C00BA7311D0BA750FD00ED00101BC51300A46
:100B6C00F2E0BC51310AF2E0BC51320AF1E0BC5166
:100B7C00330AF0E0F1D7BC6B0101BD4BBE2B010E6B
:100B8C00BB6F200E046E000E056EBDC100F0BEC121
:100B9C0001F0D4EC00F008C000F009C001F0000E28
:100BAC00011802E1000E001802E153EC01F0BAA1A9
:100BBC0041D03FC1C7F140C1C8F13B0EC96F010E16
:100BCC00CA6FE5DC00C03FF101C040F1BDC1C7F107
:100BDC00BEC1C8F139C1C9F13AC1CAF1E9EC01F0A1
:100BEC00BF6BC06B000EC05D02E1050EBF5D16E26F
:100BFC00BF513925E96EC0513A21EA6EEECF01F0B2
:100C0C000150200A08E1BF513925E16EC0513A214B
:100C1C00E26E300EE66EBF4BC02BE4D73FC1C7F17E
:100C2C0040C1C8F139C1C9F13AC1CAF1D7DCBAA780
:100C3C0001D02CDC0101BAA326D03FC1C7F140C1C1
:100C4C00C8F1340EC96F010ECA6FA1DCC76BCBECB7
:100C5C0001F000C097F101C098F100C0C7F101C0CC
:100C6C00C8F139C1C9F13AC1CAF1E9EC01F03FC18F
:100C7C00C7F140C1C8F139C1C9F13AC1CAF1AEDC02
:100C8C00BAA701D003DC0101BB6BB96BD36BD46B7E
:100C9C0041EC00F0B9C100F00036009000C080FFBC
:100CAC00800E0101B919006E800E080A005C03E287
:100CBC008098808A02D08088809A620E0C6E650EB5
:100CCC000D6E01010D2EFDD70C2EFBD70000000080
:100CDC00BAA514D0B9C100F0000EB9BFFF0E016E59
:100CEC00003600900136990E0024E96E010E0120A9
:100CFC00EA6EEECF97F1EECF98F105D0D8DC00C0BC
:100D0C0097F101C098F197C1C7F198C1C8F13FC1E3
:100D1C00C9F140C1CAF1E9EC01F0BF6BC06B000E28
:100D2C00C05D02E1050EBF5D16E2BF513F25E96EC5
:100D3C00C0514021EA6EEECF01F00150200A08E1CB
:100D4C00BF513F25E16EC0514021E26E300EE66E80
:100D5C00BF4BC02BE4D7010EBB6FBAA702D04CEC33
:100D6C0002F0800E0101B919006E800E080A005CB9
:100D7C0005E2D36BB9C1D4F141EC00F0800E070A47
:100D8C00006E800E0101B919005C07E2300ED36FC2
:100D9C00080EB95DD46F41EC00F00101BB6B3FC193
:100DAC00C7F140C1C8F1030EC96F010ECA6FCDEC7B
:100DBC0002F0800EB919006E800E0A0A005C08E27F
:100DCC003FC1E1FF40C1E2FF300EB925E66E07D00E
:100DDC003FC1E1FF40C1E2FF260EB925E66E4CECA7
:100DEC0002F097C1C7F198C1C8F13FC1C9F140C128
:100DFC00CAF1E9EC01F04CEC02F0010E0101BB6F01
:100E0C00B92B800EB919006E800E100A005CD8A0A8
:100E1C0041D7BAA704D00A0ECE6F76EC00F081BE93
:100E2C0002D0818E01D0819E0101BA5303E0010EE4
:0E0E3C00006E01D0006A00C0BAF17DD6FFD76B
:10119A0010EE15F06F0E006E020E016E2A0EF66E3C
:0E11AA00100EF76E000EF86E55EC03F01200FA
:100E4A00000000000000005F000000070007001417
:100E5A007F147F14242A7F2A1223130864623649D6
:100E6A005522500005030000001C224100004122C7
:100E7A001C0014083E081408083E080800503000F8
:100E8A000008080808080060600000201008040232
:100E9A003E5149453E00427F400042615149462148
:100EAA0041454B311814127F1027454545393C4AB4
:100EBA004949300171090503364949493606494904
:100ECA00291E00363600000056360000081422415A
:100EDA0000141414141400412214080201510906C2
:100EEA00324979413E7E1111117E7F494949363E88
:100EFA00414141227F4141221C7F494949417F09A1
:100F0A000909013E4149497A7F0808087F00417F63
:100F1A0041002040413F017F081422417F40404068
:100F2A00407F020C027F7F0408107F3E4141413E10
:100F3A007F090909063E4151215E7F091929464662
:100F4A004949493101017F01013F4040403F1F208B
:100F5A0040201F3F4038403F63140814630708705D
:100F6A0008076151494543007F41410002040810C6
:100F7A00200041417F0004020102044040404040F9
:100F8A00000102040020545454787F4844443838FD
:100F9A0044444420384444487F3854545418087E02
:100FAA000901020C5252523E7F0804047800447D23
:100FBA0040002040443D007F1028440000417F400B
:100FCA00007C041804787C080404783844444438C3
:100FDA007C14141408081414187C7C0804040848A7
:100FEA0054545420043F4440203C4040207C1C2060
:100FFA0040201C3C4030403C44281028440C5050AF
:10100A00503C4464544C44000836410000007F00C0
:10101A000000413608001008081008784641467852
:10102A0030205374617274206C696E6B202020200A
:01103A0000B5
:10103B002D2D2D204D454E55202D2D2D2D2D2D2D6E
:01104B0000A4
:10104C00414443204348302031306269747320207E
:01105C000093
:10105D003120616666696368204EB07472616D659A
:01106D000082
:10106E0031362056616C6575727320313662697443
:02107E007300FD
:10108000332053696D756C2041443737313520204A
:01109000005F
:1010910032206166666963682041444320434830D9
:0110A100004E
:1010A200313620566F696573203136206269747358
:0110B200003D
:0210B3006A01D0
:1010B50056657273696F6E2031332F30362F31309C
:0110C500002A
:1010C600204144373731355F313645415F34303959
:0710D600366D562E43200089
:1010DD002044656C616920696E746572207472615B
:0910ED006D653D33306D532000A8
:1010F60056657273696F6E2031332F30362F31305B
:0111060000E8
:101107004144373731355F6E6F6B69615F31384600
:0111170000D7
:0311180030200084
:10111B004D656E75206166666963686167653A2027
:10112B0020303D737461727420313D4E4220203269
:0E113B003D43483020333D53696D756C2000F4
:051149004348303D00A9
:02114E007C0122
:041150004E623D00AE
:02115400410157
:101156003132333435363738393031323334353647
:101166003738393031323334353637383930313231
:09117600333435363738393000C6
:10117F007061756C666A756A6F40667265652E661A
:02118F007200EC
:081191003132333435363700EA
:020000040030CA
:0D00010022090EFF0081FF0FC007E00F4035
:00000001FF
